:0200000077285F
:08000800F000030E8301F1007A
:100010000A08F2008A01831603130C1C312883128C
:1000200003130C1C312810108E010B308F00D630BA
:100030008E00AD0A04302D06031D2C28AD014A1791
:10004000AE0A1E302E06031D2C28AE0183160313A4
:10005000C30A031D2C28C40A8312031331309000F5
:100060000C1000008312031372088A00710E8300C3
:10007000F00E700E09008A01820052344534473474
:1000800055344C344134543449344F344E34203494
:1000900041344334433455344D344D3400344934C1
:1000A00052345234433435342D3450345434313492
:1000B0003034303420344C344D34333435342034FF
:1000C0004C344D34333433343534003452346534A5
:1000D0006734313436344634383438344D3435347A
:1000E0005F343234303431343134203400348301DD
:1000F0008B018A01860185018316031307309C005A
:100100009B018C018D010030850007308600013095
:100110008100831603138D018C018B01831203135D
:10012000203084008001840A041F92288316031360
:10013000AD01BB01BC01BD01BE014030CB00CD0013
:100140000630CC00CE00DC30CF00D1000530D0002E
:10015000D20083120313CA01F31073110512861122
:10016000B301B401B501D927BC25832586253D25DA
:10017000B313B513FC248F254423F5270A229225B7
:100180003D305A23F52792254F305A23F5279225E3
:1001900066305A23F527CD010230AF00CF01313050
:1001A00090008B010B128B120B178C01831603131B
:1001B0008D018C010C14831203130A128B173D2539
:1001C0008F2544238B130A228A158B208A118B17C3
:1001D000831203134A1B0D292C24FF304D05031DE8
:1001E000F328D927DE2804304F060319FC280530F0
:1001F0004F060319FC2804291C304D060319B62AA2
:100200001D304D060319E72A2B304D060319172917
:100210002C304D06031910291C29FC25CD011C2961
:1002200003102F08FF3E031C1C29AF031C292F08B5
:10023000093C031C1C29AF0A831203132F080F3932
:1002400003194B2901302F0603195E2902302F06AE
:100250000319882903302F060319502904302F066B
:100260000319C52905302F060319172B06302F0651
:100270000319172B07302F060319DE2908302F0624
:100280000319F02909302F060319502A831203138A
:10029000CD01AF01DE280000922566305A23FF29E8
:1002A0009225CF016423BA01C830E62583160313D3
:1002B0004508B1004608B200B723FF298312031393
:1002C00092250130CF0064230130BA00C830E62502
:1002D000831603133F08B1004008B200B72383120E
:1002E0000313CA1CFF2983120313C630E6254630C8
:1002F000A125C830E625CA15831603134708B100A7
:100300004808B200B72383120313CA10CA11FF2989
:1003100092250230CF0064239E250130BA00C830F8
:10032000E625831603134108B1004208B200B21F4C
:10033000A029B209B109B10A831203130330BA002C
:10034000B723831203134A1DFF29831203130130BD
:10035000BA00C630E6254630A125C830E625CA15C4
:10036000831603134908B1004A08B200B21FBF291F
:10037000B209B109B10A831203130330BA00B723DB
:10038000831203134A11CA11FF2992250330CF00AB
:100390006423C630E6254A1CD0294E30A125D22937
:1003A0004A30A1250430BA00C830E625831603136D
:1003B0004308B1004408B200B723FF298312031396
:1003C00092250730CF006423BA01C830E625CA1150
:1003D000831603135108B1005208B200B723FF2956
:1003E00092250830CF006423C830E625CA1583164D
:1003F00003134D08B1004E08B200B723FF29831242
:100400000313BA01CD01D927DE280D307F230A302E
:100410007F2308003508F039A0000310A00CA00CC1
:10042000A00C200C83160313B100B2010A30B300F4
:10043000B4014C278312031335080F3983160313B5
:10044000B1073C30B300B4014C273108B500320885
:10045000B600831203133408F039A0000310A00C77
:10046000A00CA00C200C83160313B100B2010A30BB
:10047000B300B4014C278312031334080F398316D9
:100480000313B300B4013A273508B3003608B400AB
:100490003A273108C3003208C4008312031308004E
:1004A0008B139B250630CF00642344234424013062
:1004B0004D06031D5F2A8A1545208A11B12A003096
:1004C0004D06031D672A8A154D208A11B12A033073
:1004D0004D06031D6F2A8A1553208A11B12A023056
:1004E0004D06031D772A8A155B208A11B12A053033
:1004F0004D06031D7F2A8A1561208A11B12A043016
:100500004D06031D872A8A1569208A11B12A0730F2
:100510004D06031D8F2A8A156F208A11B12A0630D5
:100520004D06031D972A8A1577208A11B12A0930B2
:100530004D06031D9F2A8A157D208A11B12A083095
:100540004D06031DA72A8A1585208A11B12A573026
:100550004D06031D512A83120313CD01AF018B17E2
:100560000A2A83120313FC24CD01512A01304B06C1
:10057000031D172B05302F06031DC62A83160313F0
:100580004B08B1004C08B2000A30CD2A8316031381
:100590004F08B1005008B2003230B300B4013A271E
:1005A0008312031305302F06031DDD2A8316031360
:1005B0003108CB003208CC00E32A8316031331083C
:1005C000CF003208D00083120313CB01172B013068
:1005D0004B06031D172B05302F06031DF72A831624
:1005E00003134B08B1004C08B2000A30FE2A8316F0
:1005F00003134F08B1005008B2003230B300B40109
:1006000043278312031305302F06031D0E2B831679
:1006100003133108CB003208CC00142B83160313CC
:100620003108CF003208D00083120313CB018312AC
:1006300003139225CA1105302F06031D212B043008
:10064000222B0530CF0064230130BA00C830E625E4
:1006500005302F06031D342BCA15831603134B08D0
:10066000B1004C08B2003B2BCA11831603134F088C
:10067000B1005008B200B72383120313CA11E02758
:10068000BA014A13CD01DE28862539082D25370801
:100690002D2536082D252030A12535082D253A3069
:1006A000A12534082D253A30A12533082D252030E9
:1006B000A1250800A60026083B20003A0319632B59
:1006C000A125A60A5B2B08004F08A5000310A50D65
:1006D000A50DA50DA50DA601260825078312031754
:1006E0008D00831603178C130C14831203170C0848
:1006F00083120313A125A60A261E6C2B0800831261
:100700000313C5000830C7008613A427C50C0318BF
:100710008B2B86138C2B8617A427C70B862B86174B
:10072000A427A427080083160313A5003030A200D5
:10073000A30064302502031CA02BA500A20A992B5C
:100740000A302502031CA72BA500A30AA02B3030DA
:100750002507A4002208A125831603132308A12539
:10076000831603132408A12583120313080083169C
:1007700003133108AF003208B000320EF038A80081
:10078000A807E23EA900323EAB0030080F39A907A6
:10079000A907AB07E93EAA00AA07AA072F0E0F393F
:1007A000AA07AB07AA0DAB0DAB09AB0D2F080F398C
:1007B000AB07A80D0730A7000A30AB07AA03031C3C
:1007C000DD2BAA07A903031CE12BA907A803031C1F
:1007D000E52BA807A703031CE92B831203132B3077
:1007E000BA1CF52B3A1CF52B2D30A12583160313CB
:1007F0002808831203130319FF2B303E002C2030EE
:10080000A12583160313290883120313303EA12563
:100810002C30CA1D0D2C3A1DA125831603132A085E
:1008200083120313303EA1252C30CA19192C3A1D0E
:10083000A125831603132B0883120313303EA12531
:100840003A19272C6430A1254330A1250800203017
:10085000A1252030A1250800831203134A1B422C36
:10086000061C2E2C4A1B422C0618322C9330810079
:100870000B11031056240318322C8B240318322C2E
:10088000E0270800CD01080083120313061C462C44
:100890000618482C933081000B11031056240318BE
:1008A000482C8B240318482CE027080083120313DC
:1008B000563084008001840A5C300406031D5A2CE3
:1008C000D301D401563084000B1D642C85240618F6
:1008D000FA2C0B1D692C8524D30A2B3053060319DF
:1008E000792C031406180310800DD40AD41982241D
:1008F000692C0310800D800D800D800D800D800D02
:1009000003100800840AD4010800831203130B119A
:1009100025308100080056308400D501D401DE0165
:10092000DC01CB01CC01CD01CE01800DD50D800DB8
:10093000D50DD40AED245D19FA2CDD0CDC0DD501A2
:10094000800DD50D800DD50DD40AED245D19FA2C3E
:10095000DD0CCB0D0530A700D501800DD50D800D28
:10096000D50DD40A54198224ED245D19FA2CDD0C1E
:10097000CC0DA70BAC2CC0305705031DC52C822411
:10098000800D800DD40A0130DE000630A700D501AD
:10099000800DD50D800DD50DD40A54198224ED2477
:1009A0005D19FA2CDD0CCD0DA70BC72C5C1C4D1767
:1009B0005E18DB2C08000630A700D501800DD50D90
:1009C000800DD50DD40A54198224ED245D19FA2C1A
:1009D000DD0CCE0DA70BDD2C0800DD010130550626
:1009E0000319F82C023055060319F92C5D1508007F
:1009F0005D1408000314080083120313061300009B
:100A000000000000000000000000061100000000CF
:100A10000515831603130611831203138E305F2509
:100A200000305F250730A3008030AB0033308400F6
:100A3000051100000000061300000000000005156D
:100A400000002B085F2500085F25840AAB0AAB0A6B
:100A5000A30B182D0511B3010800A000A100A00EE2
:100A60000F30A00530302007A1252108A0000F304D
:100A7000A00530302007A12508000613000005114D
:100A800083160313061183120313000000000000F5
:100A90000000061100000515BF305F258316031303
:100AA00006158312031333308400722572257225D4
:100AB0007225722572257225051100000800B2000A
:100AC0000830A20006130000321C06110000321884
:100AD000061500000000000006170000B20CA20B73
:100AE000622D08000830A100061300000000800CF1
:100AF0008013061980170000061700000000A10BE4
:100B0000742D840A08000130E625CB2F1030E00058
:100B10008030E625CB272030A125E00B8B2D8030BF
:100B2000E625CB2F1030E000C030E625CB27203063
:100B3000A125E00B972DC030E625CB2F0230E6250E
:100B4000CB2F83120313DF00C4270F3086055F0805
:100B5000F03986040000051400008514B6278510BE
:100B6000B6270F3086055F0EF03986040000851425
:100B7000B6278510B6270800851000000510000074
:100B8000CB270F30860530308604831603130F30D1
:100B90000605860083120313851400008510CB27F9
:100BA000851400008510CB27851400008510D927F7
:100BB0000F3086052030860485140000851028300B
:100BC000E6250830E6250C30E6250630DF00D9277B
:100BD0000F3086055F08F03986040000051000001C
:100BE0008514000085100F3086055F0EF0398604ED
:100BF000851400008510080083120313BA01061241
:100C0000000086120000F526831603133230B3006D
:100C1000B40143270A30B300B4014C272F27310811
:100C2000C5003208C600831203130130BA0006164D
:100C300000008612F526831603133108BF00320820
:100C4000C0003D08B3003E08B4003A273108BD009B
:100C50003208BE00831203130130BA0006120000EE
:100C60008616F52683160313AA30B3000A30B400A3
:100C700043273108C1003208C2003B08B3003C08DA
:100C8000B4003A273108BB003208BC00AD0A0A3074
:100C90002D06031DF02E3108C9003208CA00BB0121
:100CA000BC013D08C7003E08C800BD01BE01AD0142
:100CB000831203134A15CA14F31C642E83160313FC
:100CC0001430B300B4016A2E83160313EC30B30062
:100CD000FF30B4004D08B1004E08B2003A27470873
:100CE000B3004808B4009227031C7B2E8312031321
:100CF0000516F3147F2E831203130512F310000060
:100D0000831603134908B3004A08B400DC30B1006D
:100D10000530B200432703108F273108B500320891
:100D2000B6004D08B1004E08B2004708B3004808AD
:100D3000B400432703108D273508B3003608B400EC
:100D40003A274F08B3005008B4003A273108B500DD
:100D50003208B600CC30B3001030B4004327031C77
:100D6000BC2EB61FB82EC730D1000030D200EB2EFB
:100D7000CC30B5001030B6003508D100B1003608CF
:100D8000D200B20083120313731DCC2E83160313FB
:100D90001430B300B401D22E83160313EC30B30029
:100DA000FF30B4003A27831203134A18DD2E83164E
:100DB00003134F08B1005008B2008316031345080F
:100DC000B3004608B4009227031CEB2E83120313D2
:100DD00086157315EF2E831203138611731100000D
:100DE000831203134A138B1708008312031305277A
:100DF000620883160313B20083120313610883167B
:100E00000313B1008312031308008B138515CB273E
:100E10000613E101E20185110000861C0D2F000080
:100E200028270430A500E20D861C62108618621483
:100E30002827A50B132F0830A500E10D861C611093
:100E4000861861142827A50B1D2F85158B17080000
:100E500000000617000000000613000008008316BB
:100E600003130310B20CB10C831603130310B20C5E
:100E7000B10C0800831603133408B2073308B10716
:100E80000318B20A0800831603133308B1023408AA
:100E9000031C340FB202080083160313B901BA0110
:100EA0001030A100B20CB10C031C5C2F3408BA073F
:100EB0003308B9070318BA0A0310B30DB40DA10B18
:100EC000522F3908B1003A08B20008008316031304
:100ED000B701B8011030A100B10DB20DB70DB80DBA
:100EE00034083802031D762F33083702031C7E2F87
:100EF0003308B7023408031CB40FB802B90DBA0D99
:100F0000A10B6C2F3A08B2003908B1000800B10DEE
:100F1000B20DB10DB20DB10DB20DB10DB20DB10DDD
:100F2000B20D0800831603133208803AB00034086B
:100F3000803A3002B0009E2F34083202031DA32FE6
:100F400033083102AF0008004330A800A80BA62FD9
:100F500008000130A8000130A9002030AA00AA0B27
:100F6000AF2FA90BAF2FA80BAF2F08000130A8009F
:100F70000130A9000530AA00AF2F0130A8000130D0
:100F8000A9001430AA00AF2F0130A8000130A90039
:100F9000C830AA00AF2F0130A8000230A900F330FA
:100FA000AA00AF2F0130A8000830A900CD30AA0058
:100FB000AF2F0130A8004F30A9000130AA00AF2F99
:100FC0000130A800C430A9000230AA00AF2F0230BF
:100FD000A8008730A9006A30AA00AF2F0430A8000B
:100FE0000E30A9003830AA00AF2F0830A800A13079
:080FF000A900DA30AA00AF2FBE
:1010000003102030AC00BF01C001C101C201C30107
:10101000BE0DBD0DBC0DBB0DC30DC20DC10DC00D70
:10102000BF0DAC0B14282F284330840024204230FD
:101030008400242041308400242040308400242077
:101040003F3084002420082803300007C400C4195E
:10105000800030300007C400C41B80000800080076
:10106000A000FE309B3E2002A00D831CFA3E201CF7
:10107000A03EA00C8A28A00001302002A00D831CF5
:10108000FA3E201CA03EA00C8A283408603C0319BC
:101090008A2834083020B4008A28340803198A28A2
:1010A0003B20B4008A283508243C03198A283508D7
:1010B0003020B5008A28350803198A283B20B5005E
:1010C0008A283608283C03198A2836083020B600BA
:1010D0008A28360803198A283B20B6008A28370850
:1010E000123C03198A2837083020B7008A283708AD
:1010F00003198A283B20B7008A283908993C03192C
:101100008A2839083020B9008A28390803198A2822
:101110003B20B9000800831203137314B508031DA4
:101120007310B408031D7310731C9D2883160313DA
:10113000C301C40183120313DF288316031343087A
:10114000B1004408B2005A30B3000030B4008A1134
:1011500043278A150000031CD8284308B10044081F
:10116000B200A430B3000130B4008A1143278A15BD
:1011700000000318BC28DC284308B1004408B20072
:10118000D030B3000230B4008A1143278A15000022
:10119000031CD8284308B1004408B2006630B300ED
:1011A0000330B4008A1143278A150000031CDC2891
:1011B000831203134A10DF28831203134A14831681
:1011C00003134308B1004408B2003C30B3000030C0
:1011D000B4008A1166278A15AE000310AE0D2E08E2
:1011E000082183160313B400AE0A2E0808218316C3
:1011F0000313B3004B08B1004C08B2008A113A2720
:101200008A153108CD003208CE008312031308007E
:101210008A150A1482070034003400340034003484
:10122000003400340034003464340034C8340134F1
:101230002C340034FA340034C8340034C834003458
:10124000C8340034C8340034FA3401342C34003447
:10125000FA340034FA340034C8340034C83400346A
:10126000C8340034FA340034FA340034FA34003428
:0A127000C834003464340034003444
:02400E00212F60
:02401000FC3F73
:1042000054342E3441346334633420343D34203408
:1042100020342034203420342034203420342034FE
:1042200054342E3441346D34623420343D342034DF
:1042300020342034203420342034203420342034DE
:1042400054342E3445347834743420343D3420349E
:1042500020342034203420342034203420342034BE
:104260005434613472346934663420342034203458
:10427000203420342034203420342034203420349E
:1042800043346F346E347334543441346D34623497
:10429000203420342034203420342034203420347E
:1042A00043346F346E347334543441346334633480
:1042B000203420342034203420342034203420345E
:1042C000523454344334203441344D344A34483425
:1042D0004D3420342B34393437343534333431349D
:1042E000433441346334633441346434613470346E
:1042F000203420342034203420342034203420341E
:10430000433461346D346234413464346134703424
:1043100020342034203420342034203420342034FD
:104320002834433429345034463472346534793473
:10433000653472342034303431342F3430343134F5
:104340002F34323430343134313420345234653403
:10435000673475346C345F34313436344634383431
:1043600038345F344D3435342E34613473346D3425
:0443700020340034C1
:00000001FF
